:020000040000FA
:0600000010EF07F01200F2
:0608000010EF07F01200EA
:06082A000100540E000065
:08083000000200002E00000090
:08083800D9CFE6FFE1CFD9FFA3
:10084000040EE126DE6ADE6ADE6ADD6ADD52DD5212
:10085000FD0EDBCF00F0FE0EDBCF01F0026A036A73
:1008600001AE02D002680368D9CFE9FFDACFEAFF10
:10087000030EEB500318E8AE02D0033408D000504A
:10088000EE5C0150EE580250EE580350EE580FE265
:100890000C0EE66EF0EC06F0E552D9CFE9FFDACFA8
:1008A000EAFFEE2A000EEE22EE22EE22D1D7040E4F
:1008B000E15C02E2E16AE552E16EE552E7CFD9FF81
:1008C00012000F0EC16E070EB46E936A816A300E6D
:1008D000926E80900F0E946EF19E1200D9CFE6FFBB
:1008E000E1CFD9FF020EE1268250020B01E0010E9A
:1008F000080DF3CF02F08250010B040DF3CF01F08D
:100900008050200B01E0010EE824006E8050100B97
:1009100001E0010E002401240224DE6EDD6ADECF38
:1009200000F0DDCF01F000C0F3FF01C0F4FF020EC4
:10093000E15C03E200D0E16AE552E16EE552E7CF07
:10094000D9FF12008092320EE66E1EEC07F0E552DF
:100950008084320EE66E1EEC07F0E5528094320E73
:10096000E66E1EEC07F0E55212008082010EE66E84
:10097000E66A62DFE552E5528084010EE66EE66AC1
:100980005BDFE552E5528094010EE66EE66A54DFC5
:10099000E552E5521200380E816ED4DF320EE66E5B
:1009A000E66A4ADFE552E552010E816ECBDF320E78
:1009B000E66EE66A41DFE552E5520D0E816EC2DF5A
:1009C000320EE66EE66A38DFE552E552060E816EBB
:1009D000B9DF320EE66EE66A2FDFE552E55212000D
:1009E000010E816EAFDF0A0EE66EE66A25DFE55284
:1009F000E5521200D9CFE6FFE1CFD9FF020E816E9A
:100A0000A1DF0A0EE66EE66A17DFE552E552FD0E3B
:100A1000DBCFE6FFFE0EDB50280DF350E552E72456
:100A2000E76EFE0EE7CFDBFFFD0EDB6AFE0EDB504E
:100A3000F36EFD0EDBCFF4FFF350F45C0BE2140E0B
:100A4000816E80DF320EE66E1EEC07F0E552FD0E81
:100A5000DB2AECD7E552E7CFD9FF1200D9CFE6FF6A
:100A6000E1CFD9FFFE0EDB50816E7FDF010EE66E17
:100A7000E66AE2DEE552E552E552E7CFD9FF120021
:100A8000D9CFE6FFE1CFD9FFFD0EDBCFE9FFFE0EA8
:100A9000DBCFEAFFEF500EE0FD0EDBCFE9FFDB2AF4
:100AA000FE0EDBCFEAFF01E3DB2AEF50E66ED6DF76
:100AB000E552EAD7E552E7CFD9FF12000001646B97
:100AC000300E926EF00E936EEF0E606F60C081FF7D
:100AD000040E616F6151000821E26051FE0BE84293
:100AE000606F60C081FF050EE66EE66AA5DEE55226
:100AF000E5528150100B09E08150200B06E0815037
:100B0000400B03E08150800B01E10AD8000164052D
:100B100002E1655104D06105616FDCD7CFD71200C7
:100B2000F00E936E81CF63F000016315626F0F0EBC
:100B30006015606F60516211606F81CF63F0F00EDD
:100B40006315626FF00E625D01E0F7D7936A06D815
:100B500066C065F00001010E646F12000001676B52
:100B6000100E675D14E26751EA6A000FE96E020E2B
:100B7000EA22EF50605D08E16751EA6A100FE96E02
:100B8000020EEA22EFCF66F06729676FE9D766C0E9
:100B900081FF640EE66EE66A4FDEE552E552120012
:100BA0000001686B070E685D1DE288DF0001696F58
:100BB0006851EA6A6A0FE96E000EEA2269C0EFFF27
:100BC0006851EA6A6A0FE96E000EEA22EF504608A1
:100BD00002E108D004D069C0E6FF40DFE552000121
:100BE000682BE0D76851EA6A6A0FE96E000EEA22C4
:100BF000EF6A12000001686B070E685D16E268512B
:100C0000EA6A6A0FE96E000EEA22EF50E66E26DF0E
:100C1000E55200016829EA6A6A0FE96E000EEA22CD
:100C2000EF5001E102D0682BE7D71200D9CFE6FFE1
:100C3000E1CFD9FFE652F250800B01E0010EDF6EEA
:100C4000F29EA69EA69CA684FE0EDB50A96EFD0E0B
:100C5000DB50A86E550EA76EAA0EA76EA682A6B28E
:100C6000FED7A694DF50E8B0F28EE8A0F29EE552DF
:100C7000E552E7CFD9FF1200D9CFE6FFE1CFD9FF88
:100C8000A69CA69EFE0EDB50A96EA680A85000D0A2
:100C9000E552E7CFD9FF120014DE80828092000176
:100CA000736B746B030E74AF02D0D89003D0735D76
:100CB000000E74590CE22A0EE66E020EE66E09D89A
:100CC000E552E5520001732B000E7423EBD7E5D7F4
:100CD0001200D9CFE6FFE1CFD9FF020EE1268084D2
:100CE0008094FD0EDB50000173250F01E96EFE0EAE
:100CF000DB50000174210F01EA6EEF50D00F006E3F
:100D0000016A00BE016800C0DEFF01C0DDFFDECF6A
:100D1000E9FFDDCFEAFF200EE926020EEA22EF50BE
:100D2000816E050EE66EE66A87DDE552E552020E3B
:100D3000E15C02E2E16AE552E16EE552E7CFD9FFFC
:020D400012009F
:0E0D42002A0EF66E080EF76E000EF86E020115
:100D50000900F550336F0900F550346F03E1336734
:100D600001D03DD00900F5502E6F0900F5502F6FCE
:100D70000900F550306F09000900F550E96E0900CF
:100D8000F550EA6E090009000900F550316F0900BD
:100D9000F550326F09000900F6CF35F2F7CF36F281
:100DA000F8CF37F22EC2F6FF2FC2F7FF30C2F8FF9E
:100DB0000201315302E1325307E00900F550EE6EB3
:100DC0003107F8E23207F9D735C2F6FF36C2F7FF2E
:100DD00037C2F8FF02013307000E345BBFD71200A1
:100DE000FF0EE350066E480E01D04C0EE76EE72E64
:100DF000FED7E76AE72EFED7062EF7D700001200CF
:100E0000000EF36E00EE00F0080E01D81200EA604A
:100E100002D0EE6AFCD7F350E9601200EE6AFCD70C
:100E200012EE40F022EE40F0F86A059CA1EC06F0CC
:0C0E300029EC07F04CEC06F0FBD7120098
:040E3C00FF0EE35072
:100E4000E84E1200000000D000D000D0E82EFAD703
:020E500012008E
:020E520012008C
:0C0E5400EEEDEBE7DEDDDBD7BEBDBBB78B
:100E60007E7D7B7730313233343536373839414205
:100E7000434445467E0CB69ECCDAFA0EFECE3830A0
:020E800033003D
:00000001FF
